:100000005BC0B3C272C071C070C06FC06EC06DC043
:100010006CC06BC06AC069C068C067C066C065C09C
:1000200064C063C062C0040309042403770077003E
:1000300077002E0073006F006B006F006C00730080
:1000400070002E00610074002E0075006100140322
:100050004D004900430052004F00500052004F0035
:1000600047001201100102000008C016E10500015E
:10007000010200010902430002010080320904006C
:1000800000010202010005240010010424020605FB
:10009000240600010524010301070583030800FF6E
:1000A00009040100020A000000070501020800001F
:1000B000070581020800000011241FBECFEDCDBF4F
:1000C00010E0A0E6B0E0EEEFF7E002C005900D9280
:1000D000A236B107D9F710E0A2E6B0E001C01D9248
:1000E000A93BB107E1F7B7D188C38ACF85B7826052
:1000F00085BF8BB780648BBF8BE480938300809334
:10010000AE008AE5809382008093AD0008951F932E
:10011000DC01162F8091AD0084FF07C08091AE00F6
:1001200098E889278093AE0003C08AE58093AD00EC
:10013000912FEFEAF0E08D9181939150E1F78FEAF2
:1001400090E0612F0ED21C5F1093AD001F910895B7
:100150001F93DC01162F8091820084FF07C08091DD
:10016000830098E889278093830003C08AE5809301
:100170008200912FE4E8F0E08D9181939150E1F7B6
:1001800084E890E0612FEDD11C5F109382001F91F5
:1001900008951F93CF93DF9360919300635067FDA1
:1001A000A1C080919000CCE0D0E0C81BD109C95615
:1001B000DF4F80918F00803118F4CE0135D18CC093
:1001C0008D3209F089C0683009F086C083EC8093D5
:1001D00077008AE5809360001092620088818076C3
:1001E00021F0CE01FED0282F65C09A8110928000A8
:1001F0008981882321F41092810022E054C0853047
:1002000019F4909394004EC08630B1F58B81813003
:1002100041F482E690E0909392008093910022E175
:1002200027C0823021F4CE01C7D0282F21C08330CF
:10023000F1F4992341F486E290E090939200809348
:10024000910024E015C0913041F48AE290E090934F
:1002500092008093910024E20BC0923041F48EE42E
:1002600090E0909392008093910024E101C020E0FF
:1002700080E4809362001EC0883021F421E086E98A
:1002800090E013C0893019F4909396000BC08A3027
:1002900011F421E008C08B3029F48BE480938300B3
:1002A0008093AE0020E080E890E0909392008093ED
:1002B000910009C02F3F39F4888187FD2E8180E8A5
:1002C0008093620006C08F81882319F48E81821783
:1002D00008F0822F8093610080919300181614F427
:1002E000109293008091600084FF58C0809161005B
:1002F0008F3F09F453C0182F893008F018E0811B94
:10030000809361008091770098E889278093770037
:10031000112391F18091620087FF08C088E790E087
:10032000612F75D0182F893098F526C02091910043
:100330003091920086FF0DC0A8E7B0E080E090E029
:10034000F901E80FF91FE491ED9301961817C1F731
:1003500008C0912FD901E8E7F0E08D918193915089
:10036000E1F71150812F90E01F5F0196820F931FDC
:10037000909392008093910088E790E0612FF1D0F4
:10038000612F6C5F6C3041F08FEF8093610004C08F
:100390008FEF809361006EE16093600094E180B321
:1003A0008C7031F49150D9F71092940010928E0015
:1003B000DF91CF911F910895FC018381813049F431
:1003C00082E690E090939200809391008091620089
:1003D000089584E790E0909392008093910083E4E5
:1003E0000895FC0180818076803279F481818132A8
:1003F00011F48FEF08959281833239F488B39170AC
:100400008E7F982B98BB80E0089580E00895FC01D2
:1004100080E8808385E281831282138214821582B0
:1004200088E0868387E00895DC0130917600262FEE
:10043000932F08C0E92FF0E0E359FF4F8D9180839F
:1004400021509F5F2223B1F7360F309376008FEF54
:10045000809393000895FF920F931F9383EF82BBC5
:100460008CE081BB26E940E757E103C0CA01019750
:10047000F1F72150D9F711BA39DE87B3816C87BB08
:100480008EE388BB8AE18DB9789482E0F82E00E48F
:1004900014E07FDE409176004423C1F12091750085
:1004A0002223A1F51092930080916D008E3E19F0E9
:1004B0003091630025C080916E0080936300F092BC
:1004C000750022C0A22FB0E0FD01E359FF4F8081EB
:1004D0008FB90EB9332361F009C0912F9A95F1F7C6
:1004E0008F5F8317D0F3689A769905C080E0F9CFC3
:1004F000689A769BFDCF8FB1AB59BF4F8C932F5F1E
:10050000241700F3209375001092760080918200EA
:1005100084FFBFCF6091750080916400862B09F441
:10052000B8CF85E690E014DE8091750088708093E6
:10053000640010927500ADCFA82FB92F80E090E035
:1005400041E050EA609530E009C02D9182279795EF
:10055000879510F084279527305EC8F36F5FA8F366
:100560000895EADF8D939D930895CF93CFB7CF93EE
:10057000C395839BE9F7839B09C0839B07C0839B3B
:1005800005C0839B03C0839B01C0A6C0DF93C091BD
:100590009000DD27C956DF4F839B02C0DF91EBCF70
:1005A0002F930F931F9300B32FEF03FB20F94F936B
:1005B0003F9310B34FEF012703FB21F93BE031C01C
:1005C0004E7F012F10B3216028C0102F4D7F226075
:1005D000000000B329C04B7F2460012F000010B33E
:1005E0002BC010B3477F28602AC04F7E00B3206124
:1005F0002CC04F7D10B320622FC04F7B00B320640E
:1006000032C0422700B349934FEF0000102713FB7D
:1006100020F910B31C70C9F1297F91F2012703FB67
:1006200021F900B3237F89F2315058F1102713FBD1
:1006300022F910B3277E79F2012703FB23F92F7CDF
:1006400081F200B3102713FB24F92F7971F200C057
:1006500010B3012703FB25F92F7359F200C000B333
:10066000102713FB26F9223040F200C010B30127F7
:1006700003FB27F9243028F64F77206810B30000D9
:10068000F9CF10E41ABF00271CC03B503195C31BA3
:10069000D04010E41ABF0881033C11F10B3401F182
:1006A00020918E001981110F1213EDCF4A81441F42
:1006B000093659F10D3211F0013E29F74F7009F05A
:1006C000042F009395003F914F911F910F912F910F
:1006D000DF91CAB7C6FD4CCFCF91CFBFCF91189550
:1006E00020919500222379F3109193001123C1F5F5
:1006F0003430C2F13093930020938F00109190001A
:100700003BE0311B309390002DC0009193000130ED
:100710003CF50AE54F7049F43091600034FD24C087
:1007200000936000C7E7D0E023C0433049F0309128
:10073000820034FD19C000938200C3E8D0E018C0E5
:100740003091AD0034FD10C00093AD00CEEAD0E092
:100750000FC02795A8F45150A9F4220F0000F9CF3B
:100760004AE503C042ED01C0432FC4E1D0E032E0CE
:1007700011B31C60939A11BB02B320E41CE05F9399
:10078000012756E002BB279520F4515021F4220F97
:10079000F9CF012756E000003B5A02BBD0F2279563
:1007A00028F4515029F4220F0000F9CF012756E018
:1007B000279502BB20F4515021F4220FF9CF0127D5
:1007C00056E02991332302BB21F6037F1091940058
:1007D000110FC651D04002BB11F010938E0010E4EF
:1007E0001ABF086011B3137F402F437F5F9100C091
:0E07F00000C002BB11BB42BB66CFF894FFCF26
:0207FE005AFFA0
:00000001FF
